******************************************************************************
             TMS320C2000 Linker PC v5.2.15                     
******************************************************************************
>> Linked Wed Sep 29 13:19:47 2021

OUTPUT FILE NAME:   <D:/project28335/Balsam_165_2021_04_12/bin/UKSSTMS320F28335.out>
ENTRY POINT SYMBOL: "_c_int00"  address: 0000b931


MEMORY CONFIGURATION

         name            origin    length      used     unused   attr    fill
----------------------  --------  ---------  --------  --------  ----  --------
PAGE 0:
  ZONE0                 00004000   00001000  00000000  00001000  RWIX
  RAML0                 00008000   00004000  00003cf6  0000030a  RWIX
  RAML4                 0000c000   00001000  0000018f  00000e71  RWIX
  ZONE6                 00100000   00100000  00000000  00100000  RWIX
  FLASHH                00300000   00008000  00000000  00008000  RWIX
  FLASHG                00308000   00008000  00000000  00008000  RWIX
  FLASHF                00310000   00008000  00000000  00008000  RWIX
  FLASHE                00318000   00008000  00000000  00008000  RWIX
  FLASHD                00320000   00008000  00000000  00008000  RWIX
  FLASHC                00328000   00008000  00000000  00008000  RWIX
  FLASHA                00338000   00007f80  00000000  00007f80  RWIX
  CSM_RSVD              0033ff80   00000076  00000000  00000076  RWIX
  BEGIN                 0033fff6   00000002  00000000  00000002  RWIX
  CSM_PWL               0033fff8   00000008  00000000  00000008  RWIX
  ADC_CAL               00380080   00000009  00000007  00000002  RWIX
  OTP                   00380400   00000400  00000000  00000400  RWIX
  IQTABLES              003fe000   00000b50  00000000  00000b50  RWIX
  IQTABLES2             003feb50   0000008c  00000000  0000008c  RWIX
  FPUTABLES             003febdc   000006a0  00000000  000006a0  RWIX
  ROM                   003ff27c   00000d44  00000000  00000d44  RWIX
  RESET                 003fffc0   00000002  00000000  00000002  RWIX
  VECTORS               003fffc2   0000003e  00000000  0000003e  RWIX

PAGE 1:
  BOOT_RSVD             00000000   00000050  00000000  00000050  RWIX
  RAMM0                 00000050   000003b0  00000000  000003b0  RWIX
  RAMM1                 00000400   00000400  000003f0  00000010  RWIX
  DEV_EMU               00000880   00000180  000000d0  000000b0  RWIX
  FLASH_REGS            00000a80   00000060  00000008  00000058  RWIX
  CSM                   00000ae0   00000010  00000010  00000000  RWIX
  ADC_MIRROR            00000b00   00000010  00000010  00000000  RWIX
  XINTF                 00000b20   00000020  0000001e  00000002  RWIX
  CPU_TIMER0            00000c00   00000008  00000008  00000000  RWIX
  CPU_TIMER1            00000c08   00000008  00000008  00000000  RWIX
  CPU_TIMER2            00000c10   00000008  00000008  00000000  RWIX
  PIE_CTRL              00000ce0   00000020  0000001a  00000006  RWIX
  PIE_VECT              00000d00   00000100  00000100  00000000  RWIX
  DMA                   00001000   00000200  000000e0  00000120  RWIX
  MCBSPA                00005000   00000040  00000025  0000001b  RWIX
  MCBSPB                00005040   00000040  00000025  0000001b  RWIX
  ECANA                 00006000   00000040  00000034  0000000c  RWIX
  ECANA_LAM             00006040   00000040  00000040  00000000  RWIX
  ECANA_MOTS            00006080   00000040  00000040  00000000  RWIX
  ECANA_MOTO            000060c0   00000040  00000040  00000000  RWIX
  ECANA_MBOX            00006100   00000100  00000100  00000000  RWIX
  ECANB                 00006200   00000040  00000034  0000000c  RWIX
  ECANB_LAM             00006240   00000040  00000040  00000000  RWIX
  ECANB_MOTS            00006280   00000040  00000040  00000000  RWIX
  ECANB_MOTO            000062c0   00000040  00000040  00000000  RWIX
  ECANB_MBOX            00006300   00000100  00000100  00000000  RWIX
  EPWM1                 00006800   00000022  00000022  00000000  RWIX
  EPWM2                 00006840   00000022  00000022  00000000  RWIX
  EPWM3                 00006880   00000022  00000022  00000000  RWIX
  EPWM4                 000068c0   00000022  00000022  00000000  RWIX
  EPWM5                 00006900   00000022  00000022  00000000  RWIX
  EPWM6                 00006940   00000022  00000022  00000000  RWIX
  ECAP1                 00006a00   00000020  00000020  00000000  RWIX
  ECAP2                 00006a20   00000020  00000020  00000000  RWIX
  ECAP3                 00006a40   00000020  00000020  00000000  RWIX
  ECAP4                 00006a60   00000020  00000020  00000000  RWIX
  ECAP5                 00006a80   00000020  00000020  00000000  RWIX
  ECAP6                 00006aa0   00000020  00000020  00000000  RWIX
  EQEP1                 00006b00   00000040  00000040  00000000  RWIX
  EQEP2                 00006b40   00000040  00000040  00000000  RWIX
  GPIOCTRL              00006f80   00000040  0000002e  00000012  RWIX
  GPIODAT               00006fc0   00000020  00000020  00000000  RWIX
  GPIOINT               00006fe0   00000020  0000000a  00000016  RWIX
  SYSTEM                00007010   00000020  00000020  00000000  RWIX
  SPIA                  00007040   00000010  00000010  00000000  RWIX
  SCIA                  00007050   00000010  00000010  00000000  RWIX
  XINTRUPT              00007070   00000010  00000010  00000000  RWIX
  ADC                   00007100   00000020  0000001e  00000002  RWIX
  SCIB                  00007750   00000010  00000010  00000000  RWIX
  SCIC                  00007770   00000010  00000010  00000000  RWIX
  I2CA                  00007900   00000040  00000022  0000001e  RWIX
  RAML5                 0000d000   00003000  00000f04  000020fc  RWIX
  ZONE7A                00200000   0000fc00  0000f000  00000c00  RWIX
  ZONE7B                0020fc00   00000400  00000000  00000400  RWIX
  FLASHB                00330000   00008000  00000000  00008000  RWIX
  CSM_PWL               0033fff8   00000008  00000008  00000000  RWIX
  PARTID                00380090   00000001  00000001  00000000  RWIX


SECTION ALLOCATION MAP

 output                                  attributes/
section   page    origin      length       input sections
--------  ----  ----------  ----------   ----------------
.pinit     0    00008000    00000000     UNINITIALIZED

.text      0    00008000    00003ac3     
                  00008000    00000d39     measure.obj (.text)
                  00008d39    0000088f     DSP2833x_SWPrioritizedDefaultIsr.obj (.text)
                  000095c8    0000051b     RS485.obj (.text)
                  00009ae3    000003a2     peripher.obj (.text)
                  00009e85    0000036a     ADC.obj (.text)
                  0000a1ef    0000033d     bios.obj (.text)
                  0000a52c    0000031e     spise2p.obj (.text)
                  0000a84a    000002af     message.obj (.text)
                  0000aaf9    00000295     main.obj (.text)
                  0000ad8e    00000224     ecan.obj (.text)
                  0000afb2    000001ce     DSP2833x_Xintf.obj (.text)
                  0000b180    000001cb     DSP2833x_SysCtrl.obj (.text)
                  0000b34b    0000019b     kanal.obj (.text)
                  0000b4e6    00000171     pulto.obj (.text)
                  0000b657    00000088     rts2800_fpu32.lib : fs_div.obj (.text)
                  0000b6df    00000083     crc16.obj (.text)
                  0000b762    00000082     tools.obj (.text)
                  0000b7e4    00000080     DAC.obj (.text)
                  0000b864    00000073     DSP2833x_CpuTimers.obj (.text)
                  0000b8d7    0000005a     DSP2833x_PieCtrl.obj (.text)
                  0000b931    00000046     rts2800_fpu32.lib : boot.obj (.text)
                  0000b977    00000034     filter_bat2.obj (.text)
                  0000b9ab    0000002a     rts2800_fpu32.lib : l_div.obj (.text)
                  0000b9d5    00000022                       : i_div.obj (.text)
                  0000b9f7    00000021                       : memcpy_ff.obj (.text)
                  0000ba18    00000020                       : sqrt.obj (.text)
                  0000ba38    0000001f     log_to_mem.obj (.text)
                  0000ba57    0000001b     rts2800_fpu32.lib : args_main.obj (.text)
                  0000ba72    00000019                       : exit.obj (.text)
                  0000ba8b    00000014     DSP2833x_Adc.obj (.text)
                  0000ba9f    00000010     DSP2833x_SWPrioritizedPieVect.obj (.text)
                  0000baaf    00000009     rts2800_fpu32.lib : _lock.obj (.text)
                  0000bab8    00000007     cntrl_adr.obj (.text)
                  0000babf    00000004     DSP2833x_usDelay.obj (.text)

.cinit     0    0000bac3    00000233     
                  0000bac3    00000103     crc16.obj (.cinit)
                  0000bbc6    00000054     measure.obj (.cinit)
                  0000bc1a    00000022     pulto.obj (.cinit)
                  0000bc3c    0000001f     spise2p.obj (.cinit)
                  0000bc5b    0000001c     ecan.obj (.cinit)
                  0000bc77    0000001b     kanal.obj (.cinit)
                  0000bc92    0000001a     peripher.obj (.cinit)
                  0000bcac    0000000c     log_to_mem.obj (.cinit)
                  0000bcb8    0000000a     rts2800_fpu32.lib : _lock.obj (.cinit)
                  0000bcc2    0000000a                       : exit.obj (.cinit)
                  0000bccc    00000008     ADC.obj (.cinit)
                  0000bcd4    00000008     RS485.obj (.cinit)
                  0000bcdc    00000008     cntrl_adr.obj (.cinit)
                  0000bce4    00000008     main.obj (.cinit)
                  0000bcec    00000004     bios.obj (.cinit)
                  0000bcf0    00000004     rts2800_fpu32.lib : errno.obj (.cinit)
                  0000bcf4    00000002     --HOLE-- [fill = 0]

.econst    0    0000c000    00000111     
                  0000c000    00000100     DSP2833x_SWPrioritizedPieVect.obj (.econst)
                  0000c100    00000008     message.obj (.econst:_$P$T0$1)
                  0000c108    00000006     message.obj (.econst:_$P$T1$2)
                  0000c10e    00000003     cntrl_adr.obj (.econst)

ramfuncs   0    0000c13c    0000002b     RUN ADDR = 0000c111
                  0000c13c    0000002b     DSP2833x_SysCtrl.obj (ramfuncs)

.switch    0    0000c168    00000028     
                  0000c168    00000028     spise2p.obj (.switch)

.adc_cal   0    00380080    00000007     NOLOAD SECTION
                  00380080    00000007     DSP2833x_ADC_cal.obj (.adc_cal)

.reset     0    003fffc0    00000002     DSECT
                  003fffc0    00000002     rts2800_fpu32.lib : boot.obj (.reset)

vectors    0    003fffc2    00000000     DSECT

.stack     1    00000400    000003f0     UNINITIALIZED
                  00000400    000003f0     --HOLE--

DevEmuRegsFile 
*          1    00000880    000000d0     UNINITIALIZED
                  00000880    000000d0     DSP2833x_GlobalVariableDefs.obj (DevEmuRegsFile)

FlashRegsFile 
*          1    00000a80    00000008     UNINITIALIZED
                  00000a80    00000008     DSP2833x_GlobalVariableDefs.obj (FlashRegsFile)

CsmRegsFile 
*          1    00000ae0    00000010     UNINITIALIZED
                  00000ae0    00000010     DSP2833x_GlobalVariableDefs.obj (CsmRegsFile)

AdcMirrorFile 
*          1    00000b00    00000010     UNINITIALIZED
                  00000b00    00000010     DSP2833x_GlobalVariableDefs.obj (AdcMirrorFile)

XintfRegsFile 
*          1    00000b20    0000001e     UNINITIALIZED
                  00000b20    0000001e     DSP2833x_GlobalVariableDefs.obj (XintfRegsFile)

CpuTimer0RegsFile 
*          1    00000c00    00000008     UNINITIALIZED
                  00000c00    00000008     DSP2833x_GlobalVariableDefs.obj (CpuTimer0RegsFile)

CpuTimer1RegsFile 
*          1    00000c08    00000008     UNINITIALIZED
                  00000c08    00000008     DSP2833x_GlobalVariableDefs.obj (CpuTimer1RegsFile)

CpuTimer2RegsFile 
*          1    00000c10    00000008     UNINITIALIZED
                  00000c10    00000008     DSP2833x_GlobalVariableDefs.obj (CpuTimer2RegsFile)

PieCtrlRegsFile 
*          1    00000ce0    0000001a     UNINITIALIZED
                  00000ce0    0000001a     DSP2833x_GlobalVariableDefs.obj (PieCtrlRegsFile)

PieVectTableFile 
*          1    00000d00    00000100     UNINITIALIZED
                  00000d00    00000100     DSP2833x_GlobalVariableDefs.obj (PieVectTableFile)

DmaRegsFile 
*          1    00001000    000000e0     UNINITIALIZED
                  00001000    000000e0     DSP2833x_GlobalVariableDefs.obj (DmaRegsFile)

McbspaRegsFile 
*          1    00005000    00000025     UNINITIALIZED
                  00005000    00000025     DSP2833x_GlobalVariableDefs.obj (McbspaRegsFile)

McbspbRegsFile 
*          1    00005040    00000025     UNINITIALIZED
                  00005040    00000025     DSP2833x_GlobalVariableDefs.obj (McbspbRegsFile)

ECanaRegsFile 
*          1    00006000    00000034     UNINITIALIZED
                  00006000    00000034     DSP2833x_GlobalVariableDefs.obj (ECanaRegsFile)

ECanaLAMRegsFile 
*          1    00006040    00000040     UNINITIALIZED
                  00006040    00000040     DSP2833x_GlobalVariableDefs.obj (ECanaLAMRegsFile)

ECanaMOTSRegsFile 
*          1    00006080    00000040     UNINITIALIZED
                  00006080    00000040     DSP2833x_GlobalVariableDefs.obj (ECanaMOTSRegsFile)

ECanaMOTORegsFile 
*          1    000060c0    00000040     UNINITIALIZED
                  000060c0    00000040     DSP2833x_GlobalVariableDefs.obj (ECanaMOTORegsFile)

ECanaMboxesFile 
*          1    00006100    00000100     UNINITIALIZED
                  00006100    00000100     DSP2833x_GlobalVariableDefs.obj (ECanaMboxesFile)

ECanbRegsFile 
*          1    00006200    00000034     UNINITIALIZED
                  00006200    00000034     DSP2833x_GlobalVariableDefs.obj (ECanbRegsFile)

ECanbLAMRegsFile 
*          1    00006240    00000040     UNINITIALIZED
                  00006240    00000040     DSP2833x_GlobalVariableDefs.obj (ECanbLAMRegsFile)

ECanbMOTSRegsFile 
*          1    00006280    00000040     UNINITIALIZED
                  00006280    00000040     DSP2833x_GlobalVariableDefs.obj (ECanbMOTSRegsFile)

ECanbMOTORegsFile 
*          1    000062c0    00000040     UNINITIALIZED
                  000062c0    00000040     DSP2833x_GlobalVariableDefs.obj (ECanbMOTORegsFile)

ECanbMboxesFile 
*          1    00006300    00000100     UNINITIALIZED
                  00006300    00000100     DSP2833x_GlobalVariableDefs.obj (ECanbMboxesFile)

EPwm1RegsFile 
*          1    00006800    00000022     UNINITIALIZED
                  00006800    00000022     DSP2833x_GlobalVariableDefs.obj (EPwm1RegsFile)

EPwm2RegsFile 
*          1    00006840    00000022     UNINITIALIZED
                  00006840    00000022     DSP2833x_GlobalVariableDefs.obj (EPwm2RegsFile)

EPwm3RegsFile 
*          1    00006880    00000022     UNINITIALIZED
                  00006880    00000022     DSP2833x_GlobalVariableDefs.obj (EPwm3RegsFile)

EPwm4RegsFile 
*          1    000068c0    00000022     UNINITIALIZED
                  000068c0    00000022     DSP2833x_GlobalVariableDefs.obj (EPwm4RegsFile)

EPwm5RegsFile 
*          1    00006900    00000022     UNINITIALIZED
                  00006900    00000022     DSP2833x_GlobalVariableDefs.obj (EPwm5RegsFile)

EPwm6RegsFile 
*          1    00006940    00000022     UNINITIALIZED
                  00006940    00000022     DSP2833x_GlobalVariableDefs.obj (EPwm6RegsFile)

ECap1RegsFile 
*          1    00006a00    00000020     UNINITIALIZED
                  00006a00    00000020     DSP2833x_GlobalVariableDefs.obj (ECap1RegsFile)

ECap2RegsFile 
*          1    00006a20    00000020     UNINITIALIZED
                  00006a20    00000020     DSP2833x_GlobalVariableDefs.obj (ECap2RegsFile)

ECap3RegsFile 
*          1    00006a40    00000020     UNINITIALIZED
                  00006a40    00000020     DSP2833x_GlobalVariableDefs.obj (ECap3RegsFile)

ECap4RegsFile 
*          1    00006a60    00000020     UNINITIALIZED
                  00006a60    00000020     DSP2833x_GlobalVariableDefs.obj (ECap4RegsFile)

ECap5RegsFile 
*          1    00006a80    00000020     UNINITIALIZED
                  00006a80    00000020     DSP2833x_GlobalVariableDefs.obj (ECap5RegsFile)

ECap6RegsFile 
*          1    00006aa0    00000020     UNINITIALIZED
                  00006aa0    00000020     DSP2833x_GlobalVariableDefs.obj (ECap6RegsFile)

EQep1RegsFile 
*          1    00006b00    00000040     UNINITIALIZED
                  00006b00    00000040     DSP2833x_GlobalVariableDefs.obj (EQep1RegsFile)

EQep2RegsFile 
*          1    00006b40    00000040     UNINITIALIZED
                  00006b40    00000040     DSP2833x_GlobalVariableDefs.obj (EQep2RegsFile)

GpioCtrlRegsFile 
*          1    00006f80    0000002e     UNINITIALIZED
                  00006f80    0000002e     DSP2833x_GlobalVariableDefs.obj (GpioCtrlRegsFile)

GpioDataRegsFile 
*          1    00006fc0    00000020     UNINITIALIZED
                  00006fc0    00000020     DSP2833x_GlobalVariableDefs.obj (GpioDataRegsFile)

GpioIntRegsFile 
*          1    00006fe0    0000000a     UNINITIALIZED
                  00006fe0    0000000a     DSP2833x_GlobalVariableDefs.obj (GpioIntRegsFile)

SysCtrlRegsFile 
*          1    00007010    00000020     UNINITIALIZED
                  00007010    00000020     DSP2833x_GlobalVariableDefs.obj (SysCtrlRegsFile)

SpiaRegsFile 
*          1    00007040    00000010     UNINITIALIZED
                  00007040    00000010     DSP2833x_GlobalVariableDefs.obj (SpiaRegsFile)

SciaRegsFile 
*          1    00007050    00000010     UNINITIALIZED
                  00007050    00000010     DSP2833x_GlobalVariableDefs.obj (SciaRegsFile)

XIntruptRegsFile 
*          1    00007070    00000010     UNINITIALIZED
                  00007070    00000010     DSP2833x_GlobalVariableDefs.obj (XIntruptRegsFile)

AdcRegsFile 
*          1    00007100    0000001e     UNINITIALIZED
                  00007100    0000001e     DSP2833x_GlobalVariableDefs.obj (AdcRegsFile)

ScibRegsFile 
*          1    00007750    00000010     UNINITIALIZED
                  00007750    00000010     DSP2833x_GlobalVariableDefs.obj (ScibRegsFile)

ScicRegsFile 
*          1    00007770    00000010     UNINITIALIZED
                  00007770    00000010     DSP2833x_GlobalVariableDefs.obj (ScicRegsFile)

I2caRegsFile 
*          1    00007900    00000022     UNINITIALIZED
                  00007900    00000022     DSP2833x_GlobalVariableDefs.obj (I2caRegsFile)

.ebss      1    0000d000    00000f04     UNINITIALIZED
                  0000d000    00000746     RS485.obj (.ebss)
                  0000d746    00000036     ADC.obj (.ebss)
                  0000d77c    00000004     cntrl_adr.obj (.ebss)
                  0000d780    000004b0     measure.obj (.ebss)
                  0000dc30    0000000e     ecan.obj (.ebss)
                  0000dc3e    00000001     bios.obj (.ebss)
                  0000dc3f    00000001     rts2800_fpu32.lib : errno.obj (.ebss)
                  0000dc40    00000141     message.obj (.ebss)
                  0000dd81    00000001     --HOLE--
                  0000dd82    0000001c     spise2p.obj (.ebss)
                  0000dd9e    00000018     DSP2833x_CpuTimers.obj (.ebss)
                  0000ddb6    00000006     DSP2833x_SysCtrl.obj (.ebss)
                  0000ddbc    00000004     rts2800_fpu32.lib : _lock.obj (.ebss)
                  0000ddc0    00000100     crc16.obj (.ebss)
                  0000dec0    00000015     kanal.obj (.ebss)
                  0000ded5    00000001     --HOLE--
                  0000ded6    0000000c     peripher.obj (.ebss)
                  0000dee2    0000000c     pulto.obj (.ebss)
                  0000deee    0000000b     log_to_mem.obj (.ebss)
                  0000def9    00000006     main.obj (.ebss)
                  0000deff    00000001     --HOLE--
                  0000df00    00000004     rts2800_fpu32.lib : exit.obj (.ebss)

.logg      1    00200000    0000f000     UNINITIALIZED
                  00200000    0000f000     log_to_mem.obj (.logg)

CsmPwlFile 
*          1    0033fff8    00000008     UNINITIALIZED
                  0033fff8    00000008     DSP2833x_GlobalVariableDefs.obj (CsmPwlFile)

PartIdRegsFile 
*          1    00380090    00000001     UNINITIALIZED
                  00380090    00000001     DSP2833x_GlobalVariableDefs.obj (PartIdRegsFile)


GLOBAL SYMBOLS: SORTED ALPHABETICALLY BY Name 

address    name
--------   ----
00008000   .text
0000ba72   C$$EXIT
0000b657   FS$$DIV
0000b9d5   I$$DIV
0000b9e6   I$$MOD
0000b9ab   L$$DIV
0000b9ba   L$$MOD
0000b9c8   UL$$DIV
0000b9cf   UL$$MOD
00008e94   _ADCINT_ISR
00380080   _ADC_cal
0000c10e   _ADDR_ANSWER
0000d77c   _ADDR_FOR_ALL
0000c10f   _ADDR_TERMINAL
00000b00   _AdcMirror
00007100   _AdcRegs
0000b82e   _Anal_output
0000a26b   _Answer
0000ae55   _CAN_send
0000aee5   _CANa_handler
0000af42   _CANa_reset_err
0000af98   _CANb_handler
0000afa5   _CANb_reset_err
0000d77d   _CNTRL_ADDR
0000c110   _CNTRL_ADDR_UNIVERSAL
0000d778   _COUNT_WAIT_ONE_CANAL
0000d7f0   _Caliber_time
0000d781   _CanGO
0000d780   _CanPowse
0000dc3c   _CanTimeOutErrorTR
0000b8b5   _ConfigCpuTimer
0000d776   _ConversionCount
0000dd9e   _CpuTimer0
00000c00   _CpuTimer0Regs
0000dda6   _CpuTimer1
00000c08   _CpuTimer1Regs
0000ddae   _CpuTimer2
00000c10   _CpuTimer2Regs
0033fff8   _CsmPwl
00000ae0   _CsmRegs
0000b300   _CsmUnlock
0000d7f1   _Curr_Edge
000086d7   _Current_count
0000dedb   _Currentoz
00008d53   _DATALOG_ISR
0000b34b   _DCLK
00009263   _DINTCH1_ISR
00009284   _DINTCH2_ISR
000092a5   _DINTCH3_ISR
000092c6   _DINTCH4_ISR
000092e7   _DINTCH5_ISR
00009308   _DINTCH6_ISR
0000b357   _DOUT
0000babf   _DSP28x_usDelay
0000dcc1   _DataAnalog1
0000dcc6   _DataAnalog2
0000a84a   _Default_params
0000ded7   _Desk
00000880   _DevEmuRegs
0000b1a1   _DisableDog
00001000   _DmaRegs
00009437   _ECAN0INTA_ISR
0000947d   _ECAN0INTB_ISR
0000945a   _ECAN1INTA_ISR
0000949e   _ECAN1INTB_ISR
0000908d   _ECAP1_INT_ISR
000090ae   _ECAP2_INT_ISR
000090d1   _ECAP3_INT_ISR
000090f2   _ECAP4_INT_ISR
00009113   _ECAP5_INT_ISR
00009134   _ECAP6_INT_ISR
00006040   _ECanaLAMRegs
000060c0   _ECanaMOTORegs
00006080   _ECanaMOTSRegs
00006100   _ECanaMboxes
00006000   _ECanaRegs
00006240   _ECanbLAMRegs
000062c0   _ECanbMOTORegs
00006280   _ECanbMOTSRegs
00006300   _ECanbMboxes
00006200   _ECanbRegs
00006a00   _ECap1Regs
00006a20   _ECap2Regs
00006a40   _ECap3Regs
00006a60   _ECap4Regs
00006a80   _ECap5Regs
00006aa0   _ECap6Regs
00008d6d   _EMUINT_ISR
00008fc1   _EPWM1_INT_ISR
00008ef9   _EPWM1_TZINT_ISR
00008fe2   _EPWM2_INT_ISR
00008f1a   _EPWM2_TZINT_ISR
00009005   _EPWM3_INT_ISR
00008f3b   _EPWM3_TZINT_ISR
00009028   _EPWM4_INT_ISR
00008f5c   _EPWM4_TZINT_ISR
00009049   _EPWM5_INT_ISR
00008f7f   _EPWM5_TZINT_ISR
0000906a   _EPWM6_INT_ISR
00008fa0   _EPWM6_TZINT_ISR
00006800   _EPwm1Regs
00006840   _EPwm2Regs
00006880   _EPwm3Regs
000068c0   _EPwm4Regs
00006900   _EPwm5Regs
00006940   _EPwm6Regs
00009155   _EQEP1_INT_ISR
00009176   _EQEP2_INT_ISR
00006b00   _EQep1Regs
00006b40   _EQep2Regs
0000b926   _EnableInterrupts
0000dc30   _ErrorCount
00000a80   _FlashRegs
00006f80   _GpioCtrlRegs
00006fc0   _GpioDataRegs
00006fe0   _GpioIntRegs
0000ddba   _HSPCLK
0000aea4   _Handlai
0000932b   _I2CINT1A_ISR
0000934e   _I2CINT2A_ISR
00007900   _I2caRegs
00008d83   _ILLEGAL_ISR
00008d39   _INT13_ISR
00008d46   _INT14_ISR
000095b4   _INT_NOTUSED_ISR
0000dedc   _INcount0
0000dede   _INcount1
0000ba8b   _InitAdc
0000ad8e   _InitCan
0000b864   _InitCpuTimers
0000c111   _InitFlash
0000b238   _InitPeripheralClocks
0000b8d7   _InitPieCtrl
0000ba9f   _InitPieVectTable
0000b1a9   _InitPll
0000a5da   _InitSeeprom
0000b180   _InitSysCtrl
0000afb2   _InitXintf
0000b0d4   _InitXintf16Gpio
0000b04f   _InitXintf32Gpio
0000b829   _Init_DAC
000085a1   _Init_packMask
0000833d   _Init_sensors
00008514   _Init_sensors_more
0000d7f2   _K100
0000d7f4   _K_50
0000d7f6   _K_T1
0000d7f8   _K_T2
0000dee0   _KeyPressed
0000ddb8   _LSPCLK
00009587   _LUF_ISR
00009566   _LVF_ISR
0000a9a8   _Load_params
0000def0   _Log
0000dee2   _Lonely
0000921f   _MRINTA_ISR
000091dd   _MRINTB_ISR
00009240   _MXINTA_ISR
000091fe   _MXINTB_ISR
0000d782   _Maska
00005000   _McbspaRegs
00005040   _McbspbRegs
0000dc32   _MessageReceivedCount
0000dc34   _MessageTransivedCount
0000dcc2   _Modbus
0000ded6   _Mode
00008d78   _NMI_ISR
000095aa   _PIE_RESERVED
00380090   _PartIdRegs
00000ce0   _PieCtrlRegs
00000d00   _PieVectTable
0000c000   _PieVectTableInit
00008bf0   _Power_count
0000d7a2   _READY
0000b363   _RESET
000095c8   _RSA_RX_Handler
00009660   _RSA_TX_Handler
00009615   _RSB_RX_Handler
000096ab   _RSB_TX_Handler
0000999c   _RS_BSend
0000d700   _RS_Len
000096f6   _RS_RX_Handler
00009941   _RS_Send
00009922   _RS_SetBitMode
00009ab0   _RS_SetLineMode
000099c9   _RS_SetLineSpeed
0000984f   _RS_TX_Handler
00008d60   _RTOSINT_ISR
0000c167   _RamfuncsLoadEnd
0000c13c   _RamfuncsLoadStart
0000c111   _RamfuncsRunStart
0000aa28   _ReceiveCommandModbus3
0000aacc   _ReceiveCommandModbus6
000093b1   _SCIRXINTA_ISR
000093f5   _SCIRXINTB_ISR
0000936f   _SCIRXINTC_ISR
000093d4   _SCITXINTA_ISR
00009416   _SCITXINTB_ISR
00009390   _SCITXINTC_ISR
0000b376   _SENDBIT
00008e12   _SEQ1INT_ISR
00008e33   _SEQ2INT_ISR
00009199   _SPIRXINTA_ISR
0000a654   _SPISE2P_DRV_csclr
0000a64f   _SPISE2P_DRV_csset
0000a603   _SPISE2P_DRV_init
0000a69f   _SPISE2P_DRV_tick
000091ba   _SPITXINTA_ISR
0000d7a6   _STOPpowse
0000ddb6   _SYSCLKOUT
0000aa02   _Save_params
00007050   _SciaRegs
00007750   _ScibRegs
00007770   _ScicRegs
0000a583   _Seeprom_read
0000a52c   _Seeprom_write
0000b189   _ServiceDog
00007040   _SpiaRegs
00007010   _SysCtrlRegs
00008eb5   _TINT0_ISR
0000d792   _TPL_CANS
000089c5   _Temper_count
0000ded8   _TermoAD
0000ded9   _TermoRS
0000deda   _TermoSW
0000dc36   _TestMbox1
0000dc38   _TestMbox2
0000dc3a   _TestMbox3
00008df1   _USER10_ISR
00008dfc   _USER11_ISR
00008e07   _USER12_ISR
00008d8e   _USER1_ISR
00008d99   _USER2_ISR
00008da4   _USER3_ISR
00008daf   _USER4_ISR
00008dba   _USER5_ISR
00008dc5   _USER6_ISR
00008dd0   _USER7_ISR
00008ddb   _USER8_ISR
00008de6   _USER9_ISR
00008ed8   _WAKEINT_ISR
0000d7a4   _WAKEpowse
00008e54   _XINT1_ISR
00008e75   _XINT2_ISR
000094bf   _XINT3_ISR
000094e0   _XINT4_ISR
00009501   _XINT5_ISR
00009522   _XINT6_ISR
00009543   _XINT7_ISR
00007070   _XIntruptRegs
00000b20   _XintfRegs
000007f0   __STACK_END
000003f0   __STACK_SIZE
00000001   __TI_args_main
ffffffff   ___binit__
ffffffff   ___c_args__
0000bac3   ___cinit__
0000bac3   ___etext__
0000b9f7   ___memcpy_ff
ffffffff   ___pinit__
00008000   ___text__
0000ba57   __args_main
0000df00   __cleanup_ptr
0000df02   __dtors_ptr
0000ddbe   __lock
0000bab7   __nop
0000bab3   __register_lock
0000baaf   __register_unlock
00000400   __stack
0000ddbc   __unlock
0000ba72   _abort
0000d880   _adc_filter
0000a06a   _adc_isr
0000d746   _adc_table_lem
0000d756   _adc_table_tpl
0000b931   _c_int00
0000d794   _cal_addr
0000801e   _calc_temper_koef
0000dd9a   _ccc
0000d799   _chk
0000ba38   _clear_mem
00009add   _clear_timer_rs_live
0000d7ec   _cntCur
0000d77e   _cntr_addr_c
0000d77f   _cntr_addr_c_all
000086a4   _control_ADC
0000b51a   _cpu_timer1_isr_PULT
00008081   _cpu_timer1_isr_SENS
0000a667   _cpu_timer2_isr
0000ddc0   _crc_16_tab
000099e9   _create_uart_vars
0000d862   _curK
0000b7e4   _dOUT
0000b7f7   _dSEND
0000d850   _def_FILTERBAT
0000dec0   _digits
0000d800   _din_count
0000806b   _er_anal
0000d7a8   _err_count
0000dc3f   _errno
0000ba74   _exit
0000a4b7   _extendbios
0000b977   _filterbat
0000dc3e   _flag_DEBUG
0000def8   _flog
00009ca3   _get_Buttons
00009ae3   _get_Mode
0000a1f5   _get_command
0000b71e   _get_crc16
0000b6df   _get_crc_16
0000b6f3   _get_crc_16b
00008000   _im_calc
0000a2ba   _init
0000b762   _init_zone7
0000a2bb   _initload
0000dee7   _isBrit
0000dee6   _isLamp
0000dee4   _isMask
0000dee8   _isNumb
0000b384   _kanal_Send
0000d7b4   _lev_count
0000a2fe   _load
00200000   _logs_block
0000ab26   _main
00008d0c   _measure_all
0000dc40   _modbus
0000deef   _never_write
0000deee   _no_write
0000da40   _out_filter
0000dcc4   _outputs
0000dd00   _param
0000b7d0   _pause_us
0000a348   _peek
0000d796   _period_blink
0000d797   _period_dac
0000d795   _period_ready
0000a3c8   _poke
0000d840   _powK
0000d7e8   _preCur
0000dee9   _quaLamp
0000a1ef   _read_memory
0000ded0   _readr
00008659   _reset_errs
0000d000   _rs_a
0000d380   _rs_b
000095be   _rsvd_ISR
0000a347   _run
00009bf4   _select_tpl_canal
0000dc00   _sens_count
0000dcc8   _sens_error
0000dcca   _sens_hi_edge
0000dccc   _sens_lo_edge
0000d7d8   _sens_pair
0000d7c8   _sens_type
0000bab8   _set_cntrl_addr
00009e85   _setup_adc
000098ca   _setup_arr_cmd_length
0000b7bc   _setup_leds_line
000099f5   _setup_uart
0000d79a   _sig
0000a659   _spiSe2pFree
0000a663   _spiSe2pRead
0000a65f   _spiSe2pWrite
0000ba18   _sqrt
00009ae2   _test_rs_live
0000a4b6   _tflash
0000d79c   _time_1_5sec
0000d79e   _time_5msec
0000d7a0   _time_5sec
0000d798   _time_dac
0000aaf9   _timer_Init
0000d793   _tpl_cans
0000a409   _upload
0000dc3d   _wait
0000b7f0   _wast
0000b4e6   _what_is
0000a1f2   _write_memory
0000a4b5   _xflash
0000d7c0   _zer_count
ffffffff   binit
0000bac3   cinit
0000bac3   etext
ffffffff   pinit


GLOBAL SYMBOLS: SORTED BY Symbol Address 

address    name
--------   ----
00000001   __TI_args_main
000003f0   __STACK_SIZE
00000400   __stack
000007f0   __STACK_END
00000880   _DevEmuRegs
00000a80   _FlashRegs
00000ae0   _CsmRegs
00000b00   _AdcMirror
00000b20   _XintfRegs
00000c00   _CpuTimer0Regs
00000c08   _CpuTimer1Regs
00000c10   _CpuTimer2Regs
00000ce0   _PieCtrlRegs
00000d00   _PieVectTable
00001000   _DmaRegs
00005000   _McbspaRegs
00005040   _McbspbRegs
00006000   _ECanaRegs
00006040   _ECanaLAMRegs
00006080   _ECanaMOTSRegs
000060c0   _ECanaMOTORegs
00006100   _ECanaMboxes
00006200   _ECanbRegs
00006240   _ECanbLAMRegs
00006280   _ECanbMOTSRegs
000062c0   _ECanbMOTORegs
00006300   _ECanbMboxes
00006800   _EPwm1Regs
00006840   _EPwm2Regs
00006880   _EPwm3Regs
000068c0   _EPwm4Regs
00006900   _EPwm5Regs
00006940   _EPwm6Regs
00006a00   _ECap1Regs
00006a20   _ECap2Regs
00006a40   _ECap3Regs
00006a60   _ECap4Regs
00006a80   _ECap5Regs
00006aa0   _ECap6Regs
00006b00   _EQep1Regs
00006b40   _EQep2Regs
00006f80   _GpioCtrlRegs
00006fc0   _GpioDataRegs
00006fe0   _GpioIntRegs
00007010   _SysCtrlRegs
00007040   _SpiaRegs
00007050   _SciaRegs
00007070   _XIntruptRegs
00007100   _AdcRegs
00007750   _ScibRegs
00007770   _ScicRegs
00007900   _I2caRegs
00008000   .text
00008000   ___text__
00008000   _im_calc
0000801e   _calc_temper_koef
0000806b   _er_anal
00008081   _cpu_timer1_isr_SENS
0000833d   _Init_sensors
00008514   _Init_sensors_more
000085a1   _Init_packMask
00008659   _reset_errs
000086a4   _control_ADC
000086d7   _Current_count
000089c5   _Temper_count
00008bf0   _Power_count
00008d0c   _measure_all
00008d39   _INT13_ISR
00008d46   _INT14_ISR
00008d53   _DATALOG_ISR
00008d60   _RTOSINT_ISR
00008d6d   _EMUINT_ISR
00008d78   _NMI_ISR
00008d83   _ILLEGAL_ISR
00008d8e   _USER1_ISR
00008d99   _USER2_ISR
00008da4   _USER3_ISR
00008daf   _USER4_ISR
00008dba   _USER5_ISR
00008dc5   _USER6_ISR
00008dd0   _USER7_ISR
00008ddb   _USER8_ISR
00008de6   _USER9_ISR
00008df1   _USER10_ISR
00008dfc   _USER11_ISR
00008e07   _USER12_ISR
00008e12   _SEQ1INT_ISR
00008e33   _SEQ2INT_ISR
00008e54   _XINT1_ISR
00008e75   _XINT2_ISR
00008e94   _ADCINT_ISR
00008eb5   _TINT0_ISR
00008ed8   _WAKEINT_ISR
00008ef9   _EPWM1_TZINT_ISR
00008f1a   _EPWM2_TZINT_ISR
00008f3b   _EPWM3_TZINT_ISR
00008f5c   _EPWM4_TZINT_ISR
00008f7f   _EPWM5_TZINT_ISR
00008fa0   _EPWM6_TZINT_ISR
00008fc1   _EPWM1_INT_ISR
00008fe2   _EPWM2_INT_ISR
00009005   _EPWM3_INT_ISR
00009028   _EPWM4_INT_ISR
00009049   _EPWM5_INT_ISR
0000906a   _EPWM6_INT_ISR
0000908d   _ECAP1_INT_ISR
000090ae   _ECAP2_INT_ISR
000090d1   _ECAP3_INT_ISR
000090f2   _ECAP4_INT_ISR
00009113   _ECAP5_INT_ISR
00009134   _ECAP6_INT_ISR
00009155   _EQEP1_INT_ISR
00009176   _EQEP2_INT_ISR
00009199   _SPIRXINTA_ISR
000091ba   _SPITXINTA_ISR
000091dd   _MRINTB_ISR
000091fe   _MXINTB_ISR
0000921f   _MRINTA_ISR
00009240   _MXINTA_ISR
00009263   _DINTCH1_ISR
00009284   _DINTCH2_ISR
000092a5   _DINTCH3_ISR
000092c6   _DINTCH4_ISR
000092e7   _DINTCH5_ISR
00009308   _DINTCH6_ISR
0000932b   _I2CINT1A_ISR
0000934e   _I2CINT2A_ISR
0000936f   _SCIRXINTC_ISR
00009390   _SCITXINTC_ISR
000093b1   _SCIRXINTA_ISR
000093d4   _SCITXINTA_ISR
000093f5   _SCIRXINTB_ISR
00009416   _SCITXINTB_ISR
00009437   _ECAN0INTA_ISR
0000945a   _ECAN1INTA_ISR
0000947d   _ECAN0INTB_ISR
0000949e   _ECAN1INTB_ISR
000094bf   _XINT3_ISR
000094e0   _XINT4_ISR
00009501   _XINT5_ISR
00009522   _XINT6_ISR
00009543   _XINT7_ISR
00009566   _LVF_ISR
00009587   _LUF_ISR
000095aa   _PIE_RESERVED
000095b4   _INT_NOTUSED_ISR
000095be   _rsvd_ISR
000095c8   _RSA_RX_Handler
00009615   _RSB_RX_Handler
00009660   _RSA_TX_Handler
000096ab   _RSB_TX_Handler
000096f6   _RS_RX_Handler
0000984f   _RS_TX_Handler
000098ca   _setup_arr_cmd_length
00009922   _RS_SetBitMode
00009941   _RS_Send
0000999c   _RS_BSend
000099c9   _RS_SetLineSpeed
000099e9   _create_uart_vars
000099f5   _setup_uart
00009ab0   _RS_SetLineMode
00009add   _clear_timer_rs_live
00009ae2   _test_rs_live
00009ae3   _get_Mode
00009bf4   _select_tpl_canal
00009ca3   _get_Buttons
00009e85   _setup_adc
0000a06a   _adc_isr
0000a1ef   _read_memory
0000a1f2   _write_memory
0000a1f5   _get_command
0000a26b   _Answer
0000a2ba   _init
0000a2bb   _initload
0000a2fe   _load
0000a347   _run
0000a348   _peek
0000a3c8   _poke
0000a409   _upload
0000a4b5   _xflash
0000a4b6   _tflash
0000a4b7   _extendbios
0000a52c   _Seeprom_write
0000a583   _Seeprom_read
0000a5da   _InitSeeprom
0000a603   _SPISE2P_DRV_init
0000a64f   _SPISE2P_DRV_csset
0000a654   _SPISE2P_DRV_csclr
0000a659   _spiSe2pFree
0000a65f   _spiSe2pWrite
0000a663   _spiSe2pRead
0000a667   _cpu_timer2_isr
0000a69f   _SPISE2P_DRV_tick
0000a84a   _Default_params
0000a9a8   _Load_params
0000aa02   _Save_params
0000aa28   _ReceiveCommandModbus3
0000aacc   _ReceiveCommandModbus6
0000aaf9   _timer_Init
0000ab26   _main
0000ad8e   _InitCan
0000ae55   _CAN_send
0000aea4   _Handlai
0000aee5   _CANa_handler
0000af42   _CANa_reset_err
0000af98   _CANb_handler
0000afa5   _CANb_reset_err
0000afb2   _InitXintf
0000b04f   _InitXintf32Gpio
0000b0d4   _InitXintf16Gpio
0000b180   _InitSysCtrl
0000b189   _ServiceDog
0000b1a1   _DisableDog
0000b1a9   _InitPll
0000b238   _InitPeripheralClocks
0000b300   _CsmUnlock
0000b34b   _DCLK
0000b357   _DOUT
0000b363   _RESET
0000b376   _SENDBIT
0000b384   _kanal_Send
0000b4e6   _what_is
0000b51a   _cpu_timer1_isr_PULT
0000b657   FS$$DIV
0000b6df   _get_crc_16
0000b6f3   _get_crc_16b
0000b71e   _get_crc16
0000b762   _init_zone7
0000b7bc   _setup_leds_line
0000b7d0   _pause_us
0000b7e4   _dOUT
0000b7f0   _wast
0000b7f7   _dSEND
0000b829   _Init_DAC
0000b82e   _Anal_output
0000b864   _InitCpuTimers
0000b8b5   _ConfigCpuTimer
0000b8d7   _InitPieCtrl
0000b926   _EnableInterrupts
0000b931   _c_int00
0000b977   _filterbat
0000b9ab   L$$DIV
0000b9ba   L$$MOD
0000b9c8   UL$$DIV
0000b9cf   UL$$MOD
0000b9d5   I$$DIV
0000b9e6   I$$MOD
0000b9f7   ___memcpy_ff
0000ba18   _sqrt
0000ba38   _clear_mem
0000ba57   __args_main
0000ba72   C$$EXIT
0000ba72   _abort
0000ba74   _exit
0000ba8b   _InitAdc
0000ba9f   _InitPieVectTable
0000baaf   __register_unlock
0000bab3   __register_lock
0000bab7   __nop
0000bab8   _set_cntrl_addr
0000babf   _DSP28x_usDelay
0000bac3   ___cinit__
0000bac3   ___etext__
0000bac3   cinit
0000bac3   etext
0000c000   _PieVectTableInit
0000c10e   _ADDR_ANSWER
0000c10f   _ADDR_TERMINAL
0000c110   _CNTRL_ADDR_UNIVERSAL
0000c111   _InitFlash
0000c111   _RamfuncsRunStart
0000c13c   _RamfuncsLoadStart
0000c167   _RamfuncsLoadEnd
0000d000   _rs_a
0000d380   _rs_b
0000d700   _RS_Len
0000d746   _adc_table_lem
0000d756   _adc_table_tpl
0000d776   _ConversionCount
0000d778   _COUNT_WAIT_ONE_CANAL
0000d77c   _ADDR_FOR_ALL
0000d77d   _CNTRL_ADDR
0000d77e   _cntr_addr_c
0000d77f   _cntr_addr_c_all
0000d780   _CanPowse
0000d781   _CanGO
0000d782   _Maska
0000d792   _TPL_CANS
0000d793   _tpl_cans
0000d794   _cal_addr
0000d795   _period_ready
0000d796   _period_blink
0000d797   _period_dac
0000d798   _time_dac
0000d799   _chk
0000d79a   _sig
0000d79c   _time_1_5sec
0000d79e   _time_5msec
0000d7a0   _time_5sec
0000d7a2   _READY
0000d7a4   _WAKEpowse
0000d7a6   _STOPpowse
0000d7a8   _err_count
0000d7b4   _lev_count
0000d7c0   _zer_count
0000d7c8   _sens_type
0000d7d8   _sens_pair
0000d7e8   _preCur
0000d7ec   _cntCur
0000d7f0   _Caliber_time
0000d7f1   _Curr_Edge
0000d7f2   _K100
0000d7f4   _K_50
0000d7f6   _K_T1
0000d7f8   _K_T2
0000d800   _din_count
0000d840   _powK
0000d850   _def_FILTERBAT
0000d862   _curK
0000d880   _adc_filter
0000da40   _out_filter
0000dc00   _sens_count
0000dc30   _ErrorCount
0000dc32   _MessageReceivedCount
0000dc34   _MessageTransivedCount
0000dc36   _TestMbox1
0000dc38   _TestMbox2
0000dc3a   _TestMbox3
0000dc3c   _CanTimeOutErrorTR
0000dc3d   _wait
0000dc3e   _flag_DEBUG
0000dc3f   _errno
0000dc40   _modbus
0000dcc1   _DataAnalog1
0000dcc2   _Modbus
0000dcc4   _outputs
0000dcc6   _DataAnalog2
0000dcc8   _sens_error
0000dcca   _sens_hi_edge
0000dccc   _sens_lo_edge
0000dd00   _param
0000dd9a   _ccc
0000dd9e   _CpuTimer0
0000dda6   _CpuTimer1
0000ddae   _CpuTimer2
0000ddb6   _SYSCLKOUT
0000ddb8   _LSPCLK
0000ddba   _HSPCLK
0000ddbc   __unlock
0000ddbe   __lock
0000ddc0   _crc_16_tab
0000dec0   _digits
0000ded0   _readr
0000ded6   _Mode
0000ded7   _Desk
0000ded8   _TermoAD
0000ded9   _TermoRS
0000deda   _TermoSW
0000dedb   _Currentoz
0000dedc   _INcount0
0000dede   _INcount1
0000dee0   _KeyPressed
0000dee2   _Lonely
0000dee4   _isMask
0000dee6   _isLamp
0000dee7   _isBrit
0000dee8   _isNumb
0000dee9   _quaLamp
0000deee   _no_write
0000deef   _never_write
0000def0   _Log
0000def8   _flog
0000df00   __cleanup_ptr
0000df02   __dtors_ptr
00200000   _logs_block
0033fff8   _CsmPwl
00380080   _ADC_cal
00380090   _PartIdRegs
ffffffff   ___binit__
ffffffff   ___c_args__
ffffffff   ___pinit__
ffffffff   binit
ffffffff   pinit

[383 symbols]
